:020000041A00E0
:1000000000800010D501001A7901001A9136001AFB
:100010009936001A9D36001A9536001A0000000025
:100020000000000000000000000000008D01001A28
:100030009101001A000000009501001A9901001AB0
:100040009D01001A9D01001A9D01001A0000000088
:100050009D01001A9D01001A9D01001A9D01001AC0
:100060000D29001A2529001A9D01001A9D01001A68
:10007000A939001A9D01001A9D01001A9D01001A5C
:100080009D01001A9D01001A9D01001A9D01001A90
:100090009D01001A9D01001A9D01001A9D01001A80
:1000A0009D01001A9D01001A9D01001A9D01001A70
:1000B0009D01001A9D01001A9D01001A713C001A51
:1000C0009D01001A9D01001A9D01001A9D01001A50
:1000D0009D01001A9D01001A9D01001A9D01001A40
:1000E0009D01001A9D01001A9D01001A9D01001A30
:1000F00000000000000000009D01001A9D01001A90
:10010000000000009D01001A000000009D01001A7F
:100110009D01001A1861001A18010010EC0000007F
:100120001861001A00000810000000001861001A91
:1001300000000020000000001861001A008000206C
:10014000000000001861001A00C00020000000003C
:1001500000080010002B0000000008100000000044
:1001600000000020000000000080002000000000CF
:1001700000C0002000000000FEE700BFFEE700BF57
:10018000FEE700BFFEE700BFFEE700BFFEE700BFDF
:10019000FEE700BFFEE700BFFEE700BFFEE700BFCF
:1001A00052B110B404390023043350F8044B41F821
:1001B000044F9A42F8D810BC704700BF41B110B448
:1001C0000346002443F8044B1A1A9142FAD810BC93
:1001D000704700BF70B503F071FA184C184EB44266
:1001E00011D294E806000C3454F8045C002DF6D0CB
:1001F000043A0023043351F8040B42F8040F9D42E3
:10020000F8D8B442EDD30F4B9C4214D204F1080647
:1002100007339B1B23F0070310331C44002516E90A
:100220000300034621B143F8045B1A1A9142FAD83D
:100230000836A642F3D103F08BFDFEE71401001A45
:100240005001001A7801001A064A9369906923F058
:100250000201814218BF9161024A23F003039361B6
:10026000704700BF00000540024A936923F0010374
:100270009361704700000540024A536C43F001034C
:100280005364704700000540024A536C23F0010399
:100290005364704700000540024B186C00F00100E9
:1002A000704700BF00000540800000F1804000F56D
:1002B000A0201129836C0CD0013A090641EA820181
:1002C00023F0F85341F4006123F03D030B438364B2
:1002D000704743F001038364704700BF044B123042
:1002E00053F82000C30754BFC0F3046011207047C7
:1002F00000000540034B123053F82000C0F3830088
:10030000704700BF00000540102821D8DFE800F04A
:100310001D090B0B1120090D20172020191B151387
:100320000F000C4870470C4870470C487047042079
:10033000F4E00B4870470320F0E00220EEE000F00C
:10034000B7B80020EAE00120E8E04FF40040704731
:1003500000207047001BB70040787D0100389C1CCE
:10036000002D3101F8B50C460746FFF7CDFF1D4AB9
:100370001D4D536C1D4E23F0F85304FB00F043EA6F
:100380000763A84204F1FF3106EA030616D8B5EB6D
:10039000400F25D3002202235B0000FB03F4AC4294
:1003A00002F10102F8D9130246EA014242F040028A
:1003B0001A430C4B22F001025A64F8BD0C4B9842D0
:1003C00008D846EA0142074B42F0C00222F001027F
:1003D0005A64F8BD536C43F0010353640020F8BD28
:1003E0000023E1E700000540FF5E4C093DCC00FF23
:1003F000FFCF12132DE9F04114461F460D468046EB
:10040000FFF782FF631C0AD0B4FBF0F101FB00F39D
:100410009D421ED9C218954201F101062DD9B5FBA6
:10042000F0F4B7FBF0F6DFF884E0002104FB00F203
:1004300000E00134AA4205D3BA4203D8531E7345E3
:1004400098BF2146B4420244F3D389B90846BDE8B7
:10045000F081DFF854E07345DCD89F42DAD3C2184C
:10046000954201F1010601D872450AD9002BD6D078
:100470004046BDE8F041FFF775BF0B4B9A42CED81E
:1004800000239742F2D35BB1002AF1D0E31A121B8A
:100490009342EDD831464046BDE8F041FFF762BFD8
:1004A000002AF7D1BBE700BF00CB280CFFCA280CFD
:1004B00030B5184D6C6C83B0C4F30360FFF724FFB4
:1004C000154B014618680190286C10F0010019D0F6
:1004D000C4F3012302AA1344A20942EAD412C4F3CA
:1004E0000740D207C4F3013413F8045C04F101049B
:1004F00000F1010308D4B1FBF4F46800B3FBF0F0A1
:1005000004FB00F003B030BDB1FBF4F003FB00F0DE
:1005100003B030BD00000540C85D001A800000F146
:10052000804303F5A02310B5986C9C6CC20754BFA0
:10053000C0F304601120FFF7E7FEC4F38304013425
:10054000B0FBF4F010BD00BF1B2802D91120FFF74B
:10055000DBBE054B800003445868C307F6D4C0F3E4
:100560000460FFF7D1BE00BF5800054030B48400DE
:1005700004F1804404F5A0241B28E56D0ED8112950
:100580000AD0094828400AB140F400600BB140F09D
:10059000010040EA0160E06530BC704745F00105AC
:1005A000E56530BC704700BFFEF7FFE030B40C4C8F
:1005B00085002C441B28646806D9112401200C7086
:1005C000187030BC10707047C4F30465C4F3C020C9
:1005D00004F001040D7010701C7030BC704700BF37
:1005E000580005401B2808D8800000F1804000F525
:1005F000A020C36D23F00103C36570471B2808D8F2
:10060000800000F1804000F5A020C36D43F001039D
:10061000C36570471B2808D8054B80000344586801
:1006200000F0010080F0010070470020704700BF1B
:10063000580005401B2801D911207047044B800049
:1006400003445868C307F7D4C0F30460704700BF81
:100650005800054000290CBF012103210AB141F0D7
:100660000401022B08BF41F02001B0F5917F04D8AE
:100670002030054B43F8301070476FF481731844F5
:10068000024B43F830107047001005400020054031
:10069000B0F5917F0BD8C00000F1804000F5A2209A
:1006A000D0F8003143F00103C0F800317047044B2B
:1006B000C00003441A6842F001021A60704700BF8C
:1006C000E8170540B0F5917F0BD8C00000F18040DD
:1006D00000F5A220D0F8003123F00103C0F800316A
:1006E0007047044BC00003441A6822F001021A60EC
:1006F000704700BFE81705400249034A01230B6019
:100700001360704700100540002005400249034A6D
:1007100000230B6013607047001005400020054067
:10072000B0F5917F10B521D96FF48172144B821806
:1007300053F8324014F0010320D0124B0A221988DA
:1007400081420DD8598881420AD31046FFF7FCFE3A
:1007500014F0E00F14BF02230123B0FBF3F010BD2F
:100760009A7A1C2A03F10603E9D1EEE7064B00F161
:10077000200253F8324014F00103DED1184610BDB8
:1007800000200540CC5D001A00100540F0B492E84E
:10079000E0000B0103F1804404F5A02445EA006069
:1007A00001296662A762206202D1024DD368EB6321
:1007B000F0BC704700000540000100F1804000F5EA
:1007C000A020036A23F0010303627047000100F1D7
:1007D000804000F5A020036A43F0010303627047E4
:1007E000000100F1804000F5A020C069704700BF03
:1007F00000EB810000F5005023B9036823EA0202F0
:100800000260704703681A430260704738B5124BA4
:100810009842044618D003F58053984217D003F548
:100820007C33984215D00D48032584420CBFA2208A
:100830008120012319461A46FFF70CFF294620465E
:10084000BDE8384000F04ABA00258120F1E70125D3
:10085000FBE70225F9E700BF0010084000200C402C
:10086000154B984210B514D003F5805398420446B6
:1008700017D003F57C3398421CD0032100F062FAB4
:100880000E4884420CBFA2208120BDE81040FFF733
:1008900019BF002100F056FA8120BDE81040FFF793
:1008A00011BF0121204600F04DFA8120BDE8104023
:1008B000FFF708BF0221F5E70010084000200C40B8
:1008C00038B5084B044698420CBFA22081200D4643
:1008D000FFF726FF294602462046BDE8384000F0D3
:1008E0003DBA00BF00200C400A4B98420A460BD08C
:1008F00003F5805398420AD003F57C3398420CBF2D
:100900000221032100F07CBB002100F079BB012112
:10091000F8E700BF0010084038B5054600F05AFB64
:1009200000F00E03062B04460ED000F00602042A47
:1009300016D0022B0CBF03200120E2050DD4A30525
:100940000AD540F4007038BD284600F04FFB10F087
:100950009E0F4FF00100F0D038BD40F4807038BDDC
:100960000520EAE72DE9F04182B00546FFF7D4FF04
:10097000012817D0420706464D4C16D4B30732D48F
:1009800006F48077BFB2002F67D106F40076B6B2C6
:10099000002E6CD194F81122454C1AB9002F74D155
:1009A000002E6AD102B0BDE8F081274606E0E26879
:1009B000A3680133534013F0FF0F09D10023012234
:1009C0000DF10701284600F0B3FA0028EFD1D5E772
:1009D000BB689DF807203B4483F81021BB680133B6
:1009E000DBB2BB60EAE700220121284600F0DCFA16
:1009F000284600F0FFFA0128FAD0226863685340C5
:100A000013F0FF0F15D02A4F09E07B680133DBB2EA
:100A10007B603A687B68534013F0FF0F09D0616830
:100A20001031214400230122284600F043FA002817
:100A3000EBD122686368DFF87880534013F0FF073A
:100A40002DD13A460121284600F0AEFA88F81072FE
:100A500006F48077BFB2002F97D006F400764FF4EB
:100A600080712846B6B200F02BFB002E92D04FF4D6
:100A70000071284600F024FB8CE72846002206215E
:100A800000F092FA02B0BDE8F0810521284600F09E
:100A90008BFA012384F81132002E83D0EDE7012375
:100AA0001A461946284688F8103200F07DFA67E7A2
:100AB00000080010F8B50F46154601210022064631
:100AC000394C00F071FAFDB162682368013353407C
:100AD00013F0FF0366D0013DEDB201350021204641
:100AE00006E0426803680133534013F0FF0F57D00C
:100AF000236817F8012B234401311A74236801334A
:100B0000DBB28D422360ECD194F8103203F0FF0287
:100B1000002B34D10121304600F046FA304600F077
:100B200069FA0128FAD022686368534013F0FF0F76
:100B300015D01D4F09E07B680133DBB27B603A685A
:100B40007B68534013F0FF0F09D0616810312144D6
:100B500000230122304600F0ADF90028EBD12268D5
:100B60006368114F534013F0FF040FD13046224603
:100B7000012100F019FA87F810422846F8BD012239
:100B80003046114600F010FA2846F8BD01233046E1
:100B90001A46194687F8103200F006FA2846F8BDC2
:100BA0000D46B1E71D46AFE700080010F8B517463F
:100BB00000220C461146064600F0F6F947B31549E7
:100BC0008D68CB685D4015F0FF0518D07D1EEDB235
:100BD00001350022084605E08768C3687B4013F0B2
:100BE000FF0F13D0CB680B44013293F8103104F897
:100BF000013BCB680133DBB2AA42CB60ECD130467B
:100C00000122002100F0D0F92846F8BD1546F6E78C
:100C10003D46F4E700080010044B002283F8102240
:100C20009A60DA601A605A60704700BF00080010CE
:100C3000014B93F81102704700080010094B9842CD
:100C40000BD003F5783398420AD003F580539842CD
:100C50000CBFA4208420FFF71BBD8520FFF718BD23
:100C6000A320F8E700500840094B98420BD003F549
:100C7000783398420AD003F5805398420CBFA420E1
:100C80008420FFF71FBD8520FFF71CBDA320F8E7D8
:100C90000050084000F01F0101234009024A8B4028
:100CA00042F82030704700BF003105404009024B38
:100CB000002243F820207047003105404209064BCE
:100CC00000F01F0053F82220012303FA00F0104225
:100CD0000CBF1846002070475031054082B00723F2
:100CE000019A83604369DB0704D503680193436974
:100CF000DA07FAD403291DD8012303FA01F212F00E
:100D00000D0F05D0C36543699B06FCD50023C36561
:100D1000002301294360C3600362C3644365036524
:100D200002D10361836901934369019310238362B4
:100D300002B0704700234360C3600362C36443652D
:100D40000365F1E7032908D8012303FA01F111F043
:100D50000D0F02D00023C26DC36570472DE9F04F1F
:100D600089B0134600241B0706920025120904933C
:100D7000059223462C46DDE90467CDE900344FF0A7
:100D8000000B894607900391CDF808B04FF0FF3A69
:100D90004FF00108039D00242A46002330463946BF
:100DA00004F07CFDB0F1004F0B4688BF4B1C03F1F3
:100DB000FF31024688BF4242B1F5803F4D4409D21F
:100DC000524507D218460021CDE90001CAB1C346F9
:100DD0000294924601344445DED1039B4B4404F116
:100DE00001080393DDE904349B197C41B8F1100F2D
:100DF0001E462746CED1DDE9003423433AD0029C7B
:100E0000D846DDE90056069804EB0801A1FB05234E
:100E1000000901FB063308FB00F0002104F03EFD51
:100E200081458CBFC0EB0900C9EB0000642303FBC4
:100E300000F3B3FBF9F9B9F1020F1BD80798DDE90C
:100E40000056C368C5F30721EAB243F08003C360CC
:100E500041600260C2684FEA0813054604F00F04BF
:100E600002F07F02DBB2C26023430120AB6209B013
:100E7000BDE8F08F002009B0BDE8F08F10B4C46861
:100E80001A4304F0C00411432143C16010BC7047F1
:100E9000436913F020031ABF016001201846704710
:100EA000436913F001031DBF03680B70012018464E
:100EB000704700BF012B70B4044615D0002A34D00F
:100EC00040690B7810F020000CD00A44002001315A
:100ED0009142236000F1010004D0656911F8013BE3
:100EE000AD06F5D470BC7047FAB163694D1E9B0620
:100EF0004FF0000015F8016F11D44FF0FF33616916
:100F0000890603F1FF330CD52660002BEAD00130AF
:100F10008242E7D0636915F8016F9B06EDD5266024
:100F2000F5E7002BEBD170BC70471046DAE700BF45
:100F3000012B30B4044614D0002A32D0406910F09E
:100F400001000CD0012000E02846236801F8013B95
:100F5000824200F1010502D06369DB07F4D430BCA2
:100F60007047F2B16369DD074FF0000012D44FF013
:100F7000FF336569ED0703F1FF330ED525680D706A
:100F8000002BECD00130824201F10101E7D063690E
:100F9000DD07ECD523680B70F4E7002BE9D130BCFA
:100FA00070471046DBE700BF062996BF084B0021BB
:100FB00053F82110012A07D0426840F2073313404A
:100FC00023EA01034360704743680B434360704763
:100FD000E45D001A806840F2CF331840704700BFCC
:100FE000C36843F04003C360704700BF4069C0B2AC
:100FF000704700BF406980F04000C0F38010704728
:10100000012A0BD0032908D8012303FA01F111F0BA
:101010000D0F02D00023C26DC36570470329FCD8B1
:1010200002FA01F111F00D0FF7D0C265704700BF51
:10103000CB78022B9CBF0C4A9B184A7894BF1B7F2D
:10104000C123012A0A7808BF43F00403012A8A78E1
:1010500008BF43F00203012A08BF43F0080303F06E
:10106000CF038360704700BFE45D001A00220123B4
:101070008270C27003704370704700BF012A02D0B3
:10108000002303627047C368002243F08003C360FB
:1010900002604260C3680A7823F08003012AC360BB
:1010A00010B408BF03234FF01004846208BF03622A
:1010B0004B78012B01D010BC704705230362FAE77F
:1010C000036A19430162704710B40121002402230E
:1010D00042684460816043608368002BFCD14260B9
:1010E00010BC704710B49C1C6400A240994042EAB6
:1010F0000103C36310BC704741EA82020267704774
:101100002DE9F047B24E82B03146054601F088F82D
:1011100003F022FFAF4B53F82540D4F8AC31002B3D
:101120004AD073783278092B46D8DFE813F089006B
:10113000DC004500DC0045000A001A01450065019D
:101140006B00002A38D1A44BD4F8AC117688C4F8CF
:10115000AC1143F82520D4F87C31A04F43F00103B3
:10116000C4F87C31284600F05DFA9D499D4B9E4AAB
:10117000495D52F82500002D18BF1F4606F07F0676
:101180000F44002900F068813B789B0103449A6872
:10119000D207F6D5DB681B06F3D47306C4F85431C6
:1011A000D4F85431914A002E43F080730CBF0221D1
:1011B0000321C4F854315155D4F8AC31FBB1D4F803
:1011C000AC21854BC4F8AC21002243F82520D4F88B
:1011D0007C21824B8248834942F00102C4F87C2181
:1011E000425D002D0CBF1D460D4604F5E074AB5C5E
:1011F0005B0854F8232042F0011244F8232002B087
:10120000BDE8F087002AD7D17388DBB2012BD3D891
:101210007149D4F8AC01C4F8AC0141F82520D4F8E8
:101220007C21734E42F00102C4F87C2128463370C1
:1012300000F0F8F96D4B04225A5503F087FEBBE726
:10124000802A00F03F81822AB6D1B388654863497D
:10125000634A03F00F03002D18BF01465355C95CC4
:1012600004F5E0734908002053F82130505513F07D
:10127000011F14BF4FF0010E8646574ED4F8AC3113
:10128000C4F8AC31002746F82570D4F87C3143F01F
:101290000103C4F87C3112F80580B8F1000F40F06A
:1012A000EB8056F8252056F825305248013346F891
:1012B000253056F8257056F82530013300EB4520CF
:1012C00046F8253000F802E056F8253000F807808F
:1012D00002460121284600F011FF46F825802846E5
:1012E00000F0A0F968E7002A00F0B880022A7FF435
:1012F00063AF7288364912F0FF0F40F0ED808A88A4
:1013000012F00F013FF458AF354A032B515500F04E
:101310001C8104F5E073002D00F0158131480E5C4E
:101320007608014653F8260020F0011043F8260005
:10133000505D095C490853F8210040F0401043F823
:10134000210000235355244AD4F8AC11C4F8AC1141
:1013500042F82530D4F87C3143F00103C4F87C31E5
:10136000BDE782F08002012A3FF626AFB28871887D
:10137000D2B201AB284603F007FB00283FF41CAFB4
:10138000154FD4F8AC31C4F8AC31002647F82560CD
:10139000D4F87C31019943F001030246C4F87C3152
:1013A000284600F08BFB0E4A535D002B40F0B380C3
:1013B0000A4A0C490C4847F82530B54208BF114687
:1013C00050F82520097802EB81125386F4E600BF1D
:1013D0005C0B0010705F001A8C0B0010AC0B00103F
:1013E000880B0010C00F0010A85E001A580B0010E8
:1013F000500B0010C00B0010802A7FF4DDAE5B4E56
:10140000D4F8AC31C4F8AC31002746F82570D4F8D4
:101410007C315749574A43F00103C4F87C3111F835
:10142000058092F800E0B8F1000F57D156F825007A
:1014300056F825305049013301EB452146F8253057
:1014400001F800E00A4656F825300121284600F050
:1014500055FE46F8258042E7402397E67288D2B2CF
:10146000012A7FF4A9AEA3F103034449404AB3FA29
:1014700083F35B090B7064E7414E424956F825A09F
:1014800056F82520404B4148013246F8252056F8B1
:10149000259056F82520013246F82520002D18BF4A
:1014A0000B4600EB452C13F8081056F825300CF8C5
:1014B0000AE0624628460CF8097000F01FFE46F864
:1014C00025700CE72D4B324A1B7892F800E00BB1E7
:1014D0004EF0020E264AD0E6254A32E7284E2A4B25
:1014E00056F825C056F82510264A2848013146F8F6
:1014F0002510002D08BF1A4600EB452012F80810F1
:1015000000F80CE0024656F82530284600F0F6FDBB
:1015100046F82570E3E61C491A481E4F002D08BF07
:10152000084657F82510C35C1B4801EB831340F8AD
:1015300025605E86515DD4F87C3101228A401343D8
:10154000C4F87C3138E61048E9E60F4B0D48002D11
:1015500008BF184604F5E073415C490853F82100C0
:1015600040F0011043F82100EBE600BF8C0B0010A7
:10157000880B0010500B0010C00B0010520B001015
:10158000940B0010C00F0010AC0B001000100010E6
:10159000510B0010A85E001AA40B0010704700BF8A
:1015A0000A4B1B5C6BB170B5094B0A4D53F82030E8
:1015B0002E5C00222A54D3F8AC31044613B92E55C0
:1015C00070BD7047FFF79CFD2E5570BD580B001085
:1015D000705F001A880B001030B40B46002814BF4F
:1015E00004250625054C02E05A1C2354D3B29D4223
:1015F000FADC2154012030BC704700BF880B00107A
:1016000010B4002814BF042106210023044C00E07C
:101610002254DAB2914203F10103F9DC10BC7047A5
:10162000880B0010F8B52A4B93F90030002B0446C4
:10163000284B1FDB1D5C8DB12749284F284E294AB6
:1016400056F82030002808BF394602EB4022495D99
:1016500000F054FD002346F82430F8BD224E234A02
:1016600056F8203002EB4022012100F047FD46F8F9
:101670002450F8BD1B5C18497BB918481C4A1A4D08
:1016800052F8242045F82430002C14BF0C460446A0
:10169000217802EB81125386F8BD104D144A154E85
:1016A00052F820201448002C08BF29460025C95CA8
:1016B00046F8245002EB811250F824005586D0F8E9
:1016C0007C21012101FA03F31343C0F87C31F8BDFA
:1016D0005C0B0010880B0010C00F0010AC0B00104A
:1016E000940B0010001000108C0B0010C00B0010A9
:1016F000A85E001AA40B0010705F001A002070474B
:10170000002940D02DE9F043204B214A214C13F809
:1017100000C0214EDFF88CE0204D214F430202EB48
:10172000030883B004EB03090022BCF1000F1BD1B6
:1017300055F8203055F8204018F80330013445F8AA
:10174000204057F82040013C47F820408DF80730F2
:101750009DF807300132DBB28A428DF80730E4D1C0
:10176000002003B0BDE8F08356F8203056F8204042
:1017700019F80330013446F820405EF82040013C5F
:101780004EF82040E2E70020704700BF880B0010B1
:10179000C00B001000140010A40B00108C0B0010E4
:1017A0009C0B0010800B00102DE9F043304E314BA4
:1017B000314F324C325C54F82050002818BF1F467D
:1017C00083B017440024002A50D03B789B012B445F
:1017D000D3F808E01EF0010F2ED0DB68C3F3C0136E
:1017E00053BB29B3DFF8A0C0DFF8A0E0244F254D9C
:1017F00044029846A444A64472B955F8209055F87E
:1018000020400EF809200133621C8B4245F820204D
:101810000ED0325C002AF0D057F8204057F8202034
:101820000CF80480013301328B4247F82020F0D1BC
:10183000002003B0BDE8F0830194019BB3F57A6FFB
:1018400006D2019B01330193019BB3F57A6FF8D364
:101850000194019BB3F57A6FB5D2019B01330193DB
:10186000019BB3F57A6FF8D3002AAED14023AEE7DF
:10187000880B0010C00F0010AC0B0010A85E001AFF
:10188000940B00108C0B001000100010C00B001007
:101890002DE9F041334E344F344B354D345C002844
:1018A00014BF9E46BE4682B055F82070A64400255F
:1018B000002C55D09EF800309B013B44D3F808C063
:1018C0001CF0010F32D0DB681B062FD452B3DFF8B7
:1018D000ACC0DFF8ACE0274F274D531E420211FA8F
:1018E00083F39444013996440CE055F8208055F870
:1018F00020400EF808208B4204F1010245F8202018
:1019000010D0345C11F8012F002CEED057F8208055
:1019100057F820400CF808208B4204F1010247F8E8
:101920002020EED1002002B0BDE8F0810195019B9E
:10193000B3F57A6F06D2019B01330193019BB3F596
:101940007A6FF8D30195019BB3F57A6FB0D2019B02
:1019500001330193019BB3F57A6FF8D3002CA9D121
:101960004023AAE7880B0010AC0B0010C00F00103A
:10197000A85E001A940B00108C0B001000100010D1
:10198000C00B00107AB32DE9F041184BDFF86880E6
:10199000DFF868C01F5C164E164D541E240C43021F
:1019A00024040C44984411449C440AE055F820E077
:1019B00055F820300CF80E200133A14245F82030B4
:1019C0000ED001390A78002FF0D056F820E056F8F2
:1019D000203008F80E200133A14246F82030F0D123
:1019E0000020BDE8F0810020704700BF880B001088
:1019F000940B00108C0B001000100010C00B001096
:101A00002DE9F043254F3B5C33B9254C54F8204079
:101A10003CB90520BDE8F083224C54F82040002C4E
:101A2000F7D0C2B3DFF88890DFF888801E4EDFF869
:101A300074C01E4DDFF868E04402013A11FA82F2E8
:101A4000A1440139A044A3B955F8203055F82040ED
:101A500018F80330013445F820405EF82040013C7E
:101A60004EF8204001F8013F914214D03B5C002B1E
:101A7000EAD056F8203056F8204019F803300134E7
:101A800046F820405CF82040013C4CF8204001F82A
:101A9000013F9142EAD10020BDE8F083880B00109D
:101AA0009C0B0010800B0010A40B00108C0B00107E
:101AB00000140010C00B00100020704770B5174BC9
:101AC000DC88A2424FF0000328BF22460446FFF7FD
:101AD000DFFE134B1D5D9DB112481349134E144A8E
:101AE00056F82430002C08BF014602EB4422204661
:101AF000495D00F003FB002346F82430002070BD50
:101B00000C4E0D4A56F82430204602EB44220121A7
:101B100000F0F4FA46F82450002070BD5C0B001071
:101B2000880B0010AC0B0010C00F0010940B0010BD
:101B3000001000108C0B0010C00B0010002070472C
:101B4000F8B51F4B1F4F204E204D0446002C08BFF8
:101B50003B46305C55F82450185C05EB8010438EF2
:101B60009BB2002BFBD000232046FFF749FF335DDB
:101B7000144A63B912481649002C18BF024641F8AE
:101B80002430127805EB821500206B86F8BD0C4FCF
:101B900010481149002C18BF3A4651F82410D35C64
:101BA00005EB8315002340F824306B86305DD1F8B7
:101BB0007C21012383401343C1F87C310020F8BD10
:101BC000C00F0010AC0B0010880B0010A85E001AAC
:101BD0008C0B0010A40B0010705F001A00207047DF
:101BE000F0B50546144F1549154A164B164E1748C1
:101BF00083B000247C5540270C7014701C7002F0D8
:101C00007DF923462246214601942846009700F09C
:101C10001BFB304602F072F9284600F05FFE0C48CC
:101C200002F06CF92846012100F030FD304603B087
:101C3000BDE8F04002F062B9580B0010500B0010E4
:101C4000520B0010510B00101C5E001A045E001AAB
:101C5000285E001A38B5044610480D4602F04EF9C9
:101C60000F4B10481D5502F049F9204600F028FDA1
:101C70000D4802F043F9012D06D00C4802F03EF960
:101C80000B4B01221A7038BD0A4802F037F9204682
:101C9000FFF7A6FF084802F031F9EEE73C5E001AB4
:101CA00000180010505E001A685E001A945E001A58
:101CB000540B0010785E001A1C5E001A094A38B5F1
:101CC00001294FF00003137000D038BD05460C46C3
:101CD000194600F0DBFC21462846BDE8384000F0FC
:101CE000A7BD00BF540B0010012900D0704710B5EC
:101CF0000446054802F002F92046FFF771FF034849
:101D0000BDE8104002F0FAB8785E001A1C5E001AB6
:101D1000F8B506465B4802F0F1F85B4B5B4853F8B8
:101D20002640D4F8C03123F08013C4F8C03102F04B
:101D3000E5F8D4F8C431564823F08013C4F8C43110
:101D400002F0DCF8D4F8C831524823F08013C4F80C
:101D5000C83102F0D3F8D4F8CC314F4823F08013C7
:101D6000C4F8CC3102F0CAF8002E78D04B4802F00B
:101D7000C5F84FF0FF354A4802F0C0F8C4F8785172
:101D8000484802F0BBF80023C4F87C31464802F012
:101D9000B5F8C4F84451454802F0B0F8D4F8AC3175
:101DA000C4F8AC31424802F0A9F8D4F8BC31C4F808
:101DB000BC31404802F0A2F8D4F8B031002BFBD17E
:101DC0003D4802F09BF84FF0FF33C4F8B431D4F82B
:101DD000B451002DFBD1394802F090F8D4F84011ED
:101DE000374B384853F82670374A384B21F47F0177
:101DF000C4F84011C4F85871C4F84801C4F85451EB
:101E0000D4F85411324841F08071002E18BF1A46A0
:101E1000C4F854112B46013A8555294636B1032B97
:101E200006D802F8011F0133002EF8D1052BF8D98E
:101E3000284B294F294D2A4C2A482B4906EB4602AC
:101E400003EBC202002347F82630536145F82630E1
:101E500044F8263040F8263041F82630F8BDD4F852
:101E6000D031224823F08013C4F8D03102F046F874
:101E7000D4F8D4311E4823F08013C4F8D43102F0D2
:101E80003DF873E7C05E001A705F001AD45E001A56
:101E9000DC5E001AE45E001AEC5E001A045F001AB1
:101EA0000C5F001A205F001A285F001A305F001ACA
:101EB000385F001A405F001A505F001A605F001A16
:101EC000A85E001AC7010100AC0B0010C00F001083
:101ED000880B0010140A00109C0B00108C0B0010D3
:101EE000800B0010A40B0010940B0010F45E001A7D
:101EF000FC5E001A2DE9F04F654F664C664E674D4B
:101F000089B0002818BF3C4602900746305C55F85F
:101F100027A0205C049010F001040694604C03910B
:101F200004EB87054FEA500014BF1024002404443A
:101F30000590D5F808B000920120994600FA04F304
:101F4000DAF8B8211A40FBD11546B9F1000F00F0BC
:101F5000928009F1FF33009ACDF81CA09A46C2F393
:101F60000E02554501925C46DDF80C803AD0AEB2C7
:101F7000A6F10F07B7FA87F77F0920220021204634
:101F800003F0A6FE012362682360019BC4F8088069
:101F900063F31E426260626867F3CF326260616819
:101FA00008F5805222F47F6241F0800122F00F0296
:101FB0006160E260002D59D0DBF80020D10765D4C4
:101FC00011461268D307FBD50136B6B2B1450C6095
:101FD0000BD9102E09D00135009B554504F1200482
:101FE0009844C4D10127AEB2C7E7B9F1100FDDF8AC
:101FF0001CA040D9029A0399009D53009818294AC1
:10200000C0000E46141806EB05111150A9F110017D
:102010002561A1600298224C191802EBC10254F804
:1020200020300499C2F8149003EB81130020DA6881
:102030006FF38612DA60D968BDF800206FF3C7111C
:1020400019FB02F2D96092B2C3F808B01A8658861A
:10205000069A059B03EB0211DAF8B03101228A409F
:102060001343CAF8B03109B0BDE8F08FB9F1010FE0
:10207000B1D8DDF81CA0029A53009918094AC9008A
:102080005418002050502061A060C3E759469BE7D8
:10209000C00F0010AC0B0010880B0010705F001A0E
:1020A000A85E001A140A00100368DA0703D4184661
:1020B0001B68DA07FBD50160704700BFF8B504461E
:1020C0000D461746002120221E4603F001FE6268DD
:1020D000A56067F31E426260626866F3CF32626099
:1020E000636805F5805121F47F6143F0800321F09E
:1020F0000F0101226360E1602260F8BD2DE9F04F1D
:10210000454C464E54F820B004EB800785B011F0E2
:10211000010501954FEA5108D7F810A056F8204064
:10212000029309B214BF10250025454401204FEA4F
:1021300041198F0116460BEB070300FA05F20AEB73
:102140000905D4F8B8111140FBD120222846039389
:1021500003F0BEFD04F5E0710FFA88F0039B51F81F
:102160002020C2F38102012A4CD051F82020C2F372
:102170008142012A46D001224AF809206A68BDF846
:102180000800AE6060F31E426A606A6842F4004272
:102190006A60696806F5805222F47F6241F080012E
:1021A00022F00F026960EA6006F5005106F5405220
:1021B00006F5804621F47F6122F47F6226F47F6673
:1021C00021F00F0122F00F0226F00F0629616A614B
:1021D000AE61DA686FF38612DA60DA686FF3C712FD
:1021E000DA609D601886019BD4F8B02108EB0318D3
:1021F000012303FA08F848EA0203C4F8B03105B035
:10220000BDE8F08F4AF809205BF8071062F39F7170
:102210004BF80710B2E700BFA85E001A705F001A03
:10222000064B53F82020134653F8280F5B684B6089
:10223000CB8808600BB1002353867047A85E001A54
:1022400000487047002A00102DE9F04F80464748AB
:10225000474C50F8280054F8285089B01F1C18BF6C
:102260000127BDF8484003940E4607EB4107BC0127
:1022700000F5E0790FFA86FA2919059002910846CF
:102280000193002159F82A3004939346402203F029
:102290001FFD039A2959C2F3090262F31A41295119
:1022A0002A5942F400422A512A59049B42F0005212
:1022B0002A51029A01219160019A52BB4FEA8B0286
:1022C0001B0C02F00C041B0444F0C0048B4544EAD0
:1022D00003043AD017F00103059818BF1023D0F873
:1022E0007C2103EB570399401143C0F87C11214B2B
:1022F000214A49F82A40B8F1000F14BF9846904689
:10230000B04406B1FEB2012088F8006009B0BDE813
:10231000F08F4FEA8B4202F440249BB244F4400415
:10232000BBF1010F44EA0304E1D108A9002341F8FD
:10233000043D304649F82A20FFF782FF079B0246FA
:10234000F9B24046FFF7DAFED1E708A9019B41F850
:10235000043D304649F82A20FFF772FF4FF400731E
:102360000246F9B24046FFF7C9FEC0E7705F001AA7
:10237000A85E001AC00F0010AC0B0010704700BF21
:102380002DE9F04FDFF89CA15AF82030D3F8BC813A
:10239000C3F8BC8189B0B8F1000F69D000285E4B4A
:1023A000DFF884B100EB400914BF0422062207467F
:1023B000039203EBC90900262EE0D9F80830002B60
:1023C00040F09580C9F8143068862B8E002C4AD1D5
:1023D000524A9BB242F8273000212046FFF7CEFF39
:1023E00004F110020123934013EA080F13D05AF8A6
:1023F000273003F5E07353F82430C3F38143012BF6
:1024000068D0D9F80830002B35D1C9F814302046EF
:102410000121FFF7B3FF0136039BF4B2A34227DD8E
:10242000012000FA04F313EA080FD9D05AF8273034
:1024300003F5E07353F82430C3F3810383422FD0B4
:102440005BF82750D9F8141005EBC415EB682A8EF9
:10245000C3F30E43D31A9BB22B860029ADD16886F5
:102460002B8E002CB4D02E4A9BB242F82730B3E713
:1024700009B0BDE8F08F5BF82700B9F81020D9F853
:10248000001000EBC4100546002004959BB22D8E71
:1024900000903846FFF72EFD0498ADB20586B6E7EA
:1024A0005BF8272002EBC41208A9138ED0689AB2F9
:1024B000C0F30E43D31A41F8043D2046FFF7C0FE97
:1024C0006100024601F0FE014FF400733846FFF749
:1024D00015FE81E707A92046FFF7B2FE6100013132
:1024E0000246C9B2079B3846FFF708FE8FE7B5F8EA
:1024F00030E0D9F80010059100201FFA8EF1B9F8EC
:10250000102004919BB2009005993846FFF7F2FC29
:10251000BDF810302B8658E7140A00109C0B0010F1
:10252000800B0010705F001AA85E001A2DE9F04FB2
:102530004E4B53F82050D5F84841D5F844311C4053
:1025400085B04DD0E7070646C5F8444105D5D5F816
:10255000AC31D5F8BC31002B65D1E1033CD5D5F8C1
:102560007821D5F87C3102EA0308C5F87881B8F102
:10257000000F31D03E493F4ADFF80CA17302002E14
:10258000194414BF4FF004094FF00609039103EBFF
:10259000020B00271AE018EA030F16D0D5F8B8216D
:1025A00049001342C9B210D15AF8262002EB811219
:1025B000528E92B24AB9304A06EB460002EBC00294
:1025C000002933D05269002A40D00137F9B20123E3
:1025D000894503FA01F3DEDC22061FD4630602D428
:1025E00005B0BDE8F08F3046FFF792FB234800248A
:1025F000402502270194234622460095214687550F
:102600003046FFF721FE01940095304622462146D0
:102610008023FFF719FE05B0BDE8F08FFEF7BEFF7F
:102620006306DDD5DFE7FFF7ABFE96E7144B43F813
:102630002610D5F87C3123F00103C5F87C315A46C9
:102640004FF400733046FFF759FDBEE70D4840F8E0
:102650002620D5F87C2122EA0303C5F87C31039AB1
:102660004FF400733046FFF749FDAEE7705F001A84
:1026700000140010C00B0010140A0010580B0010BA
:102680009C0B0010800B0010A85E001A38B50446A1
:1026900009480D4601F032FC084B53F82420D2F8CB
:1026A000403125B923F00103C2F8403138BD43F071
:1026B0000103C2F8403138BD785F001A705F001A1C
:1026C00038B50546424C434801F018FC635D43B3FE
:1026D000414801F013FC414B414853F82540022387
:1026E000C4F8403101F00AFCD4F840319B07FBD418
:1026F0003C4801F003FC0223C4F8A83135B93A483C
:1027000001F0FCFB394B0922C3F8A421384801F041
:10271000F5FB2846FFF7FCFA3648BDE8384001F0E3
:10272000EDBB354801F0EAFBC5F10103E35C8BB377
:10273000DDB10320FDF756FF01231A4619466E202E
:10274000FDF788FF2D4A2E49536823F0200353607C
:102750004B5D012B36D02B4AD2F8843143F0807385
:10276000C2F8843101236355B2E7274801F0C6FB64
:102770000120FDF737FF01231A4619466520FDF7B2
:1027800069FF224801F0BAFB1C4A536823F020037A
:102790005360E7E71E4801F0B1FB1E4B1E481F497E
:1027A0001F4A586299621F481A6201F0A7FB002075
:1027B000FEF716F8C207FAD51B4801F09FFB002D63
:1027C000B7D1D2E7194B1222C3F8802CC3E700BF60
:1027D000440A0010885F001A2860001A705F001A0F
:1027E0004060001A4860001A5860001A00600040FB
:1027F0006C60001A8460001A9C5F001A003004406C
:102800000018001000700040F45F001A1060001AF9
:10281000B45F001A00000540FF030E046220300080
:102820001C000004C85F001AE05F001A0060084046
:10283000264B00280CBF4FF480724FF4007202291F
:1028400070B5C3F8802004461FD0C4F10106204DA6
:10285000AB5D23B11F4A536843F0200353606CB94A
:102860006520FDF72FFF0120FDF7C8FEAB5D13B11A
:102870000020FDF7ABFF00232B5570BD6E20FDF748
:1028800021FF0320FDF7BAFEF0E7134B53F8203089
:102890004FF0FF320021C3F84421C3F87821C3F878
:1028A0007C11D3F8AC21C3F8AC21D3F8BC21C3F818
:1028B000BC21D3F8B021002AFBD14FF0FF32C3F87E
:1028C000B421D3F8B421002AFBD1BEE700E100E037
:1028D000440A001000300440705F001A0028044BC6
:1028E0000CBF4FF480724FF400721A60704700BF43
:1028F00000E100E00028044B0CBF4FF480724FF45D
:102900000072C3F88020704700E100E0044B1A78A1
:102910001B78012B00D070470020FFF707BE00BFD7
:1029200000180010044B5A785878C0B2012800D023
:102930007047FFF7FBBD00BF0018001070B5002303
:102940000546C0F80E30C0F81230C0F8163082B01C
:10295000407B012407E06B79A3421DD06B7AA34230
:102960001FD00134E4B200280CBF06230423A34285
:102970001CDD6B78A342EED16E8829798023022278
:1029800000290CBF00210221019100962146FFF78A
:102990005BFC60B1687BE4E7EE88297A00230222C1
:1029A000EEE76E89297B80230322E9E7012002B04C
:1029B00070BD00BFF8B51E4A437BD25C042A02D02A
:1029C00002242046F8BDD0F81220002AF8D0194E73
:1029D0004278F254044608460D4603F0C7F92946EA
:1029E00082B20023607BFEF753FF677BF45D94B1F6
:1029F00011481249124D134A55F82730002F08BFCD
:102A0000014602EB4722095D38460024FFF776FBBA
:102A100045F82740D5E70C4D0C4A55F8273002EB16
:102A2000472201213846FFF769FB45F82740C8E7F0
:102A3000580B0010880B0010AC0B0010C00F0010DA
:102A4000940B0010001000108C0B0010C00B001035
:102A500070B51B4C437BE45C042C02D0022420465E
:102A600070BDD0F81240002CF8D0164D04464078C6
:102A7000E8540023607BFEF70BFF667BAC5D94B1EE
:102A800011481249124D134A55F82630002E08BF3E
:102A9000014602EB4622095D30460024FFF72EFB7B
:102AA00045F82640DBE70C4D0C4A55F8263002EB82
:102AB000462201213046FFF721FB45F82640CEE7AC
:102AC000580B0010880B0010AC0B0010C00F00104A
:102AD000940B0010001000108C0B0010C00B0010A5
:102AE0002DE9F843464A437BD25C042A03D00224F2
:102AF0002046BDE8F883D0F81220002AF7D0DFF88E
:102B00002081427808F803200546407B0E460028C5
:102B10003DD198F800403B4B1A5DD1075BD5002CA6
:102B200063D127464023384A52F8272013449A6835
:102B3000D20702D5DB681B061AD5002C3ED0314BDC
:102B40003249DFF8D090324A002808BF194602EB1C
:102B5000472259F82730095DFFF7D0FA002349F8DA
:102B60002730FEF7CBFD002847D16F7B18F80740D0
:102B7000BCB1284A264B52F8270052F8271003EB25
:102B80004723013142F827101E540024B0E718F8FB
:102B900000401E4B1A5DD10707462AD534BB40239F
:102BA000C1E71D4A1D4B52F8270052F8271003EBCE
:102BB0004723013142F827101E5499E7DFF8589057
:102BC000164A59F8273002EB47220121FFF796FAFF
:102BD00049F82740C5E70C4B1B68074603EB8212F8
:102BE000538E9BB2002BC3D1A7E707461B5D9B0109
:102BF00099E7054B53F82030F0E7044678E700BF2B
:102C0000580B0010AC0B0010A85E001AC00F00108B
:102C100000100010940B00108C0B0010C00B001063
:102C2000880B00102DE9F8434A4A437BD25C042A02
:102C300003D002242046BDE8F883D0F81220002AF1
:102C4000F7D0454F4278FA54447B3E5D66BB434B18
:102C500053F824309BB22BB3002C48D0404B9A5DE4
:102C6000D10734D43F4B53F8243003EB8212558EF6
:102C7000ADB2003518BF01258146D6B138483A4972
:102C8000DFF8F480394A58F82430002C18BF014688
:102C900002EB4422895D2046FFF730FA002348F812
:102CA00024305DB30024C5E7314B53F824309BB288
:102CB000D1E7DFF8C8802F4A58F8243002EB4422CD
:102CC00001212046FFF71AFA48F82460E9E77EBBA5
:102CD0004023244A52F8242013449D6815F001052E
:102CE000CAD0DD68C5F3C01585F00105C4E71E4BE9
:102CF0009A5DD507EBD41B4B1B68B6E7FEF7FEFCCD
:102D0000C8B999F80D60BC5DBCB1154816491A4F99
:102D1000164A57F82630002E18BF014602EB46220D
:102D2000095D3046FFF7EAF92C4647F8265081E75F
:102D30009B5D9B01CDE704467CE7104F0D4A57F899
:102D4000263002EB462201213046FFF7D7F947F83B
:102D500026506FE7580B0010880B00109C0B0010DA
:102D6000C00F0010A85E001AAC0B0010001000107D
:102D7000800B0010C00B0010940B00108C0B001087
:102D80000549427B8A5C042A00D07047D0F8123093
:102D9000002BFAD0FFF746BF580B0010294A437B9F
:102DA000D25C042A01D000207047D0F81220002AFB
:102DB000F9D0F0B424494279CA54244E437B244FBD
:102DC000CC5C2448002B14BF32463A4650F82350BE
:102DD000125D05EB8212528E92B282B194B91E4AF4
:102DE00052F8230080B290B9002B08BF3E461B4921
:102DF000327841F8230005EB8215688600E0002058
:102E0000F0BC7047164A52F8230080B218B152F84D
:102E1000230080B2F4E7002B08BF3E46114A345D20
:102E2000114F05EB841547F8230052F823406886BC
:102E3000C95CD4F87C2101238B401343C4F87C3156
:102E4000DEE700BF580B0010880B0010C00F001009
:102E5000AC0B0010A85E001A9C0B00108C0B00102D
:102E6000800B0010705F001AA40B0010584A437BBF
:102E7000D25C042A40F0A580D0F81220002A00F08D
:102E8000A0802DE9F041534D4279EA545249437BE9
:102E9000524CEA5C524E002B18BF0C4656F82310D9
:102EA000A45C01EB84111C46498E89B2002900F014
:102EB0008C8062B34B4F57F8231089B2002947D159
:102EC0009E464FF6FF7057F8231089B2E1B9434F81
:102ED000DFF8048156F82340DFF818C1BEF1000F77
:102EE0000CBF3E464646404FB25C4CF8231004EB04
:102EF000821257F823405186E95CD4F87C210123E3
:102F00008B401343C4F87C3100B2BDE8F0813749EF
:102F100051F8232092B2002A36D19E464FF6FF7018
:102F200051F8232092B2002AEED12C4C2A4F56F8A9
:102F300023102F4DBEF1000F0CBF26463E4645F82C
:102F40002320347801EB841300B25A86BDE8F08167
:102F5000284B294A53F824E053F82410013143F850
:102F6000241057F82430013B02EB442247F8243068
:102F700012F80EC090F80DE015F80E201FFA8CF034
:102F80007346E2B1174F9EE7194A1C4C52F823E0F2
:102F900052F82370013742F8237051F82320013A88
:102FA00041F8232004EB432414F80EC090F80DE000
:102FB00015F80E201FFA8CF07346002AE2D10B4957
:102FC000AEE74FF6FF7000B270474FF6FF709BE719
:102FD000580B0010880B0010C00F0010AC0B001035
:102FE000A85E001A800B0010705F001A9C0B001086
:102FF0008C0B0010A40B001000140010C00B00106C
:10300000224A437BD25C042A00D07047D0F81220B9
:10301000002AFAD070B51E4A1E4D467A5168EE5409
:10302000044682B010686B4603C308220023607B0D
:103030006946FEF72DFC04F11001607B002302229B
:10304000FEF726FC647B2D5D6DB9134E134A56F8CE
:10305000243002EB442201212046FFF74FF846F8C6
:10306000245002B070BD0E480E490F4E0F4A56F85C
:103070002430002C08BF014602EB4422495D204663
:10308000FFF73CF8002346F82430EAE7580B00101D
:103090009060001A880B00108C0B0010C00B001001
:1030A000AC0B0010C00F0010940B001000100010AB
:1030B000704700BF704700BF2DE9F84F8349427B3E
:1030C00051F82230D3F8AC4124B1814D0478AE8858
:1030D000A64201D0BDE8F88F04466878203803285E
:1030E000F8D8DFE810F020000501AD0104002978D0
:1030F000774D2129EED1D3F8AC017649C3F8AC0164
:10310000002041F82200D3F87C2142F00102C3F8EC
:103110007C21607BFEF786FA69882046C9B2FFF7FA
:10312000C9FFBDE8F88F28782128D3D1D3F8AC01A6
:10313000684DC3F8AC01002045F82200D3F87C218B
:10314000DFF8A4C1644F654EDFF8A0E142F0010250
:10315000C3F87C21627B824218BF674616F802C022
:103160005EF8223017F80C0003EB8010438E9BB200
:10317000002BFBD0BCF1000F40F0428255F82280BA
:1031800055F82270564B5748013745F8227053F8CE
:103190002270013F43F8227055F822C055F8227082
:1031A000013745F8227053F82270013F43F822702E
:1031B00055F8229055F82270013745F8227053F8DF
:1031C0002270013F43F8227055F822A055F8227072
:1031D000013745F8227053F8227000EB4220013F7E
:1031E00043F8227010F80CC010F80A2010F809708B
:1031F00010F80800637B3F0447EA0262024342EA98
:103200000C22C4F81220F25C002A40F0D58155F857
:1032100023C055F82300334A314F013045F82300CD
:1032200057F8230002EB4322013812F80C2047F82C
:103230002300637BA275F25C002A40F0B28155F84E
:1032400023C055F82300274A254F013045F82300B5
:1032500057F8230002EB4322013812F80C2047F8FC
:103260002300637BE275F25C002A40F08F8155F801
:1032700023C055F823001B4A194F013045F823009D
:1032800057F8230002EB4322013812F80C2047F8CC
:103290002300637B2276F25C002A40F05A810E48BC
:1032A000114E5EF8231045F82320002B0CBF034677
:1032B00033461B7801EB83135A86607BFEF7B2F925
:1032C0002046FFF7F5FEBDE8F88F00BF705F001ADB
:1032D0005C0B00108C0B0010AC0B0010880B001066
:1032E0009C0B0010C00B0010C00F0010A85E001A4D
:1032F0002978A1297FF4EEAED3F8AC11B44DC3F810
:10330000AC11002145F82210D3F87C21B14EDFF832
:10331000D0C2B14FDFF8E4E242F00102C3F87C21F1
:10332000617B705C5EF821E0002918BF67460744A6
:10333000002800F0A5803B789B0173449A68D2076F
:10334000F6D5DB681B06F3D4D4F81230DFB20028C0
:1033500040F0CE8055F8218055F821009F4A013079
:1033600045F8210055F821C055F82100013045F8F5
:10337000210055F821E055F82100013045F82100E1
:1033800002EB4122180A02F8087055F8219002F861
:103390000C0055F821001F0C01301B0E02F80E70B6
:1033A00045F8210002F80930637BA17DF25C002A18
:1033B00040F09080894855F8237055F8232000EBA1
:1033C00043200132C15545F82320637BE17DF25C47
:1033D000002A71D1814855F8237055F8232000EB5D
:1033E00043200132C15545F82320637B217EF25CE6
:1033F000002A53D1794855F8237055F8232000EB63
:1034000043200132C15545F82320677BF65D002E2D
:1034100038D073487049734D734A55F82730002FE0
:1034200018BF014602EB4722895D3846FEF766FE6B
:10343000002345F82730607BBDE8F84FFEF7F2B86F
:1034400029786A4D21297FF445AED3F8AC01604953
:10345000C3F8AC01002041F82200D3F87C2142F0EF
:103460000102C3F87C21607BFEF7DCF8AB78EA78D8
:1034700043EA0223E3812046FFF71AFEBDE8F88FF6
:1034800040235AE7554A55F8273002EB47220121DD
:103490003846FEF733FE45F82760CCE75148524ADC
:1034A00050F823E050F8237002EB4322013740F834
:1034B000237002F80E10A8E74A484B4A50F823E060
:1034C00050F8237002EB4322013740F8237002F8D2
:1034D0000E108AE74348444A50F823E050F823701E
:1034E00002EB4322013740F8237002F80E106CE71C
:1034F0003C4A3D4852F8219052F821E00EF1010E6D
:1035000042F821E052F8218052F821E00EF1010E3C
:1035100042F821E052F821C052F821E00EF1010EEC
:1035200000EB412042F821E000F8097052F821E058
:1035300052F821704FEA132900F8089001374FEA3A
:1035400013481B0E00F80C8042F8217000F80E3072
:103550002AE7214DDFF888C051F823705EF8230078
:10356000DFF88CE0002B0CBF294661460025895C02
:103570004EF8235000EB811101224D86F15CD7F803
:103580007C318A401343C7F87C3196E6184A194FBC
:1035900052F823C052F82300013042F82300164AA3
:1035A0006EE6134A134F52F823C052F8230001303D
:1035B00042F82300104A4BE60D4A0E4F52F823C042
:1035C00052F82300013042F823000B4A28E600BFDE
:1035D0008C0B0010880B0010AC0B0010C00B0010FF
:1035E000C00F0010940B0010001000105C0B0010B6
:1035F000A40B0010800B001000140010A85E001A2D
:103600001F4B204853F8228053F82270DFF878B01F
:10361000013743F8227050F82270013F40F82270C1
:1036200053F822C053F82270013743F8227050F843
:103630002270013F40F8227053F8229053F8227014
:10364000013743F8227050F82270013F40F8227091
:1036500053F822A053F82270013743F8227050F833
:1036600022700BEB4223013F40F8227013F80CC08C
:1036700013F80A2013F8097013F80800BAE500BF20
:10368000A40B0010800B001000140010FFFFFFFFC0
:1036900001F06CB901F06AB901F068B901F066B9DE
:1036A00008B54FF0FF3000F033FE01F01BF9024B7C
:1036B0004FF480521A6008BD00E100E02DE9F043AC
:1036C0009E4C9F4D012385B0194620464FF4804201
:1036D000FDF78EF804262046012340220021FDF745
:1036E00087F8204601234FF400620521C5F8A06148
:1036F000FDF77EF801231A4620460221FDF778F8EF
:103700000123194632462046FDF772F800F07CFB93
:1037100001231A4620460321FDF76AF820460123BB
:1037200002220321FDF764F800F076FB0123412219
:103730001946C5F8902720464FF40042FDF758F887
:10374000012244232046052184F82F204FF4807263
:10375000C5F884310023FDF74BF800F021FB00F0A1
:103760000FFBFCF771FD00230193019BB3F57A6F0A
:1037700006DA019B01330193019BB3F57A6FF8DB05
:10378000704B71491A460420FCF734FE00230122D5
:1037900009210420FCF7EAFE00230293029BB3F503
:1037A0007A6F06DA029B01330293029BB3F57A6FBC
:1037B000F8DB664B664D6449614CDFF88081654EED
:1037C0001A460420FCF716FEFCF74EFD2846FDF7CE
:1037D0001DF8EB68042243F08003EB602A60EA687E
:1037E000002340F2852102F07F02EA602846A962A8
:1037F0001A460321FDF742FB1922D123C4F8002108
:103800004FF00109C4F804310027284603A98DF8B8
:103810000E708DF80F708DF80D90FDF709FC49467C
:103820002846FDF761F80620FCF7DCFE4FF49070A7
:10383000FCF72EFF484B49491A68494842F02002DC
:103840001A601A6822F4716222F00C0242F40062DB
:1038500042F004021A604FF48062DA601122C4F868
:103860008C91C4F89C91C4F8002C4FF000620A605F
:1038700046214322C4F89410C4F8C4102260626048
:103880004222C4F8BC20C4F8C0204722C4F88023D8
:10389000C4F884234022C4F80821C4F81821C4F8CD
:1038A000B4101421C4F8B8101621C4F80C114FF04C
:1038B000106141664B4603214046C4F82873FCF76B
:1038C00097FF482388F866703046C4F82433FDF724
:1038D000B5F93046FDF7F8FB224B4FF02008CC221B
:1038E000C4F8B020C3F80080B36A43F00803B362A1
:1038F000B36AFF2243EA0803B3623260736805F5D6
:10390000804543EA090373602846FDF797F9284686
:10391000FDF7DAFB144BEB606A68144BE02142EAD6
:1039200009026A6083F81F7383F80C1383F8088315
:1039300083F8191305B0BDE8F08300BF00400F40C5
:1039400000600840805CD705002D310100B9AE0B46
:10395000001008400040084000001040AC00054046
:103960000000054004700C4000EE020000E100E0A1
:1039700008B50B4800F0C2FA00F018FA00F008FA97
:103980003820FDF787F97220FCF782FE054B4FF0D7
:10399000D852C3F804243820BDE80840FDF786B9A2
:1039A000B460001A003004402DE9F04FA44ADFF85B
:1039B000B8A2A44800238DB01362FDF785FBDAF8A6
:1039C0000430A14ADAF800000B931946136BCAF8C9
:1039D00000300AEB81011B1A8B60D16B490705D4BB
:1039E000116A01F1376101F5D8311162954A916888
:1039F00047F23052914200F28580DAF8BC10934AC7
:103A0000914D934C642000FB01F0A2FB0062801AF0
:103A100002EB5002FF2028604FF48050C4F8800170
:103A200052098748C2F164022C294362C26276D9E6
:103A300000230024CDE90834CDE90634CDE904346F
:103A4000CDE902344FF00008DFF820B2DDF82C9009
:103A5000CDF80080B9F12C0F8CBFA9F12D024A4698
:103A60000AEB82027B4B966833445B45404609F182
:103A7000010935D801F0CAFB02460B4604460D4643
:103A8000DDE9020101F076FACDE90201304601F0EC
:103A9000ADFB02460B4606460F46DDE9040101F088
:103AA00069FA3246CDE904013B462046294601F039
:103AB00013FC02460B46DDE9060101F05BFACDE995
:103AC000060108FB08F001F0A1FB009C02460B4632
:103AD0000134DDE90801009401F04CFACDE9080158
:103AE00008F10108B8F12D0FB4D1009B042B1AD8AE
:103AF0000B9B01332D2B08BF0023CAF804300DB0F7
:103B0000BDE8F08F504A52494FF48050FF241460B2
:103B1000C1F880014A48642243620021C262013137
:103B2000CAF8BC10E4E7184601F060FB04460D46F5
:103B300002460B46DDE9020101F0F8FC2246804610
:103B400089462B46DDE9040101F0F0FC4246CDE94F
:103B500000014B462046294601F0BEFB06460F46B3
:103B600002460B46DDE9000101F0B6FB02460B46BA
:103B7000DDE9060101F0FCF9324604460D463B46FC
:103B80004046494601F0A8FB02460B46DDE9080124
:103B900001F0EEF902460B462046294601F0C6FC2C
:103BA00004460D4602460B464046494601F094FB4A
:103BB00002460B46DDE9000101F0DAF900228046F9
:103BC0008946254B2046294601F086FB42464B4656
:103BD00001F0D0F9002206460F46204B2046294628
:103BE00001F07AFB42464B4601F0C4F901F036FE83
:103BF000134D1B4B0446002230463946AC6201F09F
:103C000095FC01F02BFE0F493B46C86032460AA1E5
:103C1000D1E9000101F08AFC124BC3E9060100F072
:103C200061FE18B9DAF804300B9361E700F09EFEEC
:103C3000F8E700BFAFF300800000000060E3A6419A
:103C4000100B001000500840004008406DC1166C79
:103C500000E100E0009CABF400804640004046409C
:103C600000408F4020010010480A001000983A00E0
:103C70002D4B2E492E48FF22F0B5C3F8302F4C684B
:103C8000002C2ED000232B4D80F8C0304B604FF01D
:103C90000053D0F8C410284C1C60284A59604C1CB2
:103CA000C0F8C440916899601169D960D2681A61FE
:103CB00000212348596103F1200299612A60D861EB
:103CC0002049194C02F120000B2301E011F8013DBD
:103CD000403354F8233042F8043B9042F6D1286038
:103CE000F0BD194F90F8C060124D57F826302A6881
:103CF00003F5804E724502D09342E1D1C9E701221B
:103D00005A61D1F800E0731CDBB2B240052B42EAE5
:103D10000E0280F8C0300A6012BF57F8233080F8D6
:103D2000C0404FF00053B4E700101040400B0010AB
:103D3000480A0010180100103412CDAB00500840A2
:103D4000CDAB3412B360001A9860001AAFF3008054
:103D500008B54FF0FF3000F0DBFA00F0C3FD064B72
:103D60004FF480521A6000F021F800F011F801F0D1
:103D7000C7F800F021F8FEE700E100E0FFFFFFFFD9
:103D8000024B012283F82E20704700BF00400F40F5
:103D9000024B002283F82E20704700BF00400F40E6
:103DA000014B01229A71704700400F40014B0022E5
:103DB0009A71704700400F40024B002283F8402068
:103DC000704700BF00400F40024B012283F84020A3
:103DD000704700BF00400F40024B002283F8AB2029
:103DE000704700BF00400F40024B012283F8AB2018
:103DF000704700BF00400F40024B002283F8222092
:103E0000704700BF00400F40024B012283F8222080
:103E1000704700BF00400F40034B0121002283F890
:103E2000601083F86120704700400F40034B002171
:103E3000012283F8601083F86120704700400F4032
:103E4000034B93F8A800003018BF0120704700BF53
:103E500000400F4008B5084B08485022C3F82823FB
:103E6000032140220023FCF7C3FC044A92F8663089
:103E7000002BFBD008BD00BF0060084000400F4091
:103E800008B50321012308484022FCF7B1FC06488D
:103E900064234FF00101013B80F86610024AFAD119
:103EA00082F8663008BD00BF00400F40104964230F
:103EB0004FF00002013B81F82F20FBD110B40D4AD6
:103EC0000D4C182120FA01F3DBB2A36013681B0626
:103ED000FCD5083911F1080FF4D1054964234FF0DE
:103EE0000102013B81F82F20FBD110BC704700BFBD
:103EF00000400F40040010400000104038B50A4C4C
:103F00000546012038B963699B06FCD515F8013BCD
:103F1000002BF7D138BD29780348FCF7B9FF0030F2
:103F200018BF0120EFE700BF0010084001281DD096
:103F300019D3022814D0B0F5807F1AD8802340F21C
:103F40000111DA0882EA93025A4082EA1312013020
:103F50005B0843EAC2138842DBB2F2D118467047CD
:103F600040F2022070474FF0FF30704740F20230BD
:103F700070478020704700BF012816D012D3022856
:103F80000ED0202813D8102383EA9302013002F0C8
:103F900001025B08212843EA0213F5D11846704755
:103FA000422070474FF0FF3070476220704710206A
:103FB000704700BF30B585B004AC04E90F0001982C
:103FC00001F014F900224FF07C5301F085F904460A
:103FD00000980D4601F00AF902460B462046294694
:103FE00000F0C8FF0AA3D3E9002301F075F9029B92
:103FF0000446039800FB03F00D4601F0F7F8024673
:104000000B462046294601F091FA05B030BD00BFAD
:1040100000000000D01273412DE9F04784B004ACD9
:1040200004E90F00019DDDF800A0029E039FB5F595
:10403000004F6AD2FF2E68D81F2F66D8BAF5004FFE
:1040400063D2304601F0D2F802460B4634A1D1E9E2
:10405000000101F06BFA34A3D3E9002380468946BE
:1040600001F0ACFB044600284FD14046494630A33E
:10407000D3E9002301F0C0FB804600284BD128463D
:1040800001F0B4F800224FF07C5301F025F904460A
:1040900050460D4601F0AAF802460B462046294636
:1040A00000F068FF1EA3D3E9002301F015F90446D0
:1040B00007FB06F00D4601F099F802460B46204634
:1040C000294601F033FA044678000D4601F08EF8D7
:1040D00002460B462046294601F0FEF816A3D3E916
:1040E000002304460D4601F069FB90B914A3D3E9FF
:1040F00000232046294601F07FFB4FF0010300B961
:10410000034683F00100C0B200E0002004B0BDE827
:10411000F0874046FAE72046F8E700BFAFF300809B
:1041200000000000D01273410000000080844E4166
:1041300000000000A3E1A141000000C02A64B041DA
:10414000000000C02A64C0412DE9F04F93B014462E
:104150001D46CDE906450D9065A3D3E90023204611
:10416000294600240B9401F0E1F90123CDE9000177
:104170000C93614B0A9408940994049405930C9D44
:104180004FF0010AAB4654461EE0BE46049A059B1A
:104190003046714601F012FB02960397002200237D
:1041A00068B1DDE9020101F009FB00286BD1CDF80F
:1041B0002080CDF828A0049605970B95099401342A
:1041C000B4F5807FAB446DD0584601F00FF802463D
:1041D0000B4606460F46DDE9000101F07DF800229E
:1041E000464B8046894601F0FDFA0028E7D140465B
:1041F000494601F00BFB824600F0F8FFCDE90201D1
:1042000002460B464046494600F0B2FE00223B4BB8
:1042100001F062F800223A4B00F0ACFE01F01EFB08
:10422000CDF838A00F901094119512AB804613E989
:104230000F00FFF7F1FE0028C1D0404600F0D6FF86
:1042400000224FF07C5301F047F8DDE9022300F033
:1042500091FE27A3D3E9002301F03EF832463B4606
:1042600001F064F902460B46DDE9060100F080FE2C
:104270000022002306460F4601F0BEFA002884D132
:1042800007F1004E82E70994013407F10043B4F5C9
:10429000807F04960593CDF82080CDF828A00B955B
:1042A000AB4491D104980599164B002201F086FA8F
:1042B00028B90C9B0133202B0C937FF460AF0022B4
:1042C000114B0498059901F007F801F0C7FA02466E
:1042D0000D980A9C0460089C4460099C0B4B846008
:1042E0000B9CC4609A6013B0BDE8F08FAFF3008000
:1042F00000000000D0127341000049400000E0407F
:104300000000E03F0000F03F00408F40100B001025
:10431000274A2DE9F04143F2E7038046002143F2AA
:104320008700B8F1FF3F18BF1846D51D14460E464A
:1043300041F61F7C4FF0C60E01E014F8011F1D4B23
:104340008F003B44C3F84061C3F88061C3F8C0C12B
:10435000C3F880E0186419B1196C41F40061196464
:10436000AC42EAD1B8F1FF3F134B1ED0186B4FF4AB
:10437000007140441862D96310494FF00040002397
:1043800008601946012001E012F8013F00FA03F32A
:10439000AA4241EA03014FF00103F5D1054AC2F8F0
:1043A0001C12C2F8243FBDE8F0810421D963E3E781
:1043B000CC60001A001010400040084000E100E00E
:1043C000084A094B91681962A2F55432D16A196002
:1043D00002F5242292F8A820003218BF0122DA60E8
:1043E000704700BF00500840100B0010F0B585B0BA
:1043F000024606460B4668460F46FFF7A5FE009D9F
:1044000015B9032005B0F0BD3946304601F026FA53
:10441000174E0299039A174B174F184C78600129D1
:1044200008BF3346012A14BF00200820034323633A
:104430001046FFF7A1FD06460846FFF777FD46EA5E
:104440000030A063019B0E4903EBC533E363236B8C
:1044500023F0010323632246652001E00138D1D017
:10446000D36A002BFAD00139F6D10220CAE700BF87
:104470001518000411180004100B0010000005406E
:1044800040771B0084B0F0B506AC84E80E00079EB0
:104490000A9F089C9DF830E00B9A099B0D46F60098
:1044A00006EBC53541F6C26148F2010606EBC404CD
:1044B00001EB87310A4E0560032701EB4E11446082
:1044C000C7604661BDE8F040120302EB035303F5F9
:1044D000000303F224438160036104B0704700BF0E
:1044E0000500580084B038B504AC84E80F00059886
:1044F00000F07CFE044606980D4600F077FE02466A
:104500000B462046294601F011F8044604980D4652
:1045100000F06CFE02460B462046294600F02AFDBC
:10452000044608980D4600F061FE02460B46002046
:104530000C4900F0FBFF02460B462046294600F0DE
:10454000CBFE079B0446012098400D4600F04EFE2E
:104550000B4602462946204600F0E8FFBDE83840F9
:1045600004B07047000034402DE9F04F95B0144678
:104570001D46139098A3D3E900232046294600F056
:10458000D5FF97A3D3E9002304460D46CDE90645A0
:1045900001F014F990B994A3D3E9002320462946E9
:1045A00001F00CF9002800F0D680974C002304217C
:1045B000CDE90A341A461291234607E0934C0023B2
:1045C0000521CDE90A341A4612912346DDE9060198
:1045D00000F082FE86A3D3E9002304460D4600F0D6
:1045E000A5FF01F013F9824600F000FE80A3D3E995
:1045F0000023CDE9080100F06FFE02460B4620467D
:10460000294600F0B5FC7AA3D3E9002300F08EFF21
:104610004FF0010BCDE90E014FF00009DFF80882E1
:1046200028E02846214601F0C9F80022002378B18D
:104630002846214601F0C2F8002840F0C980129BAC
:104640000D93059B0C93CDF844A01097A946A04666
:104650000136022E1ED14846414600226C4BDDF841
:1046600014B001F0ABF8002858D10BF1010BBBF5E9
:10467000805F53D0584600F0B9FD02460B46DDE995
:104680000E01CDE9002300F027FECDE9020100264E
:10469000CDF814B0304600F0B9FDDDE9022300F09A
:1046A00069FC01F0DBF8074600F0A0FDDDE900231E
:1046B00000F03CFFDDE9082300F05CFC4CA3D3E9EB
:1046C000002300F009FEDDE90A2300F02FFFDDE9F9
:1046D000062300F04DFC40A3D3E9002300F0FCFDCD
:1046E0000022002305460C4601F068F84A4643467E
:1046F000002896D004F100444A4628464346214605
:1047000001F05CF80028A3D0A946A046129B0D93A7
:10471000059B10970C93CDF844A099E700223D4BE0
:104720003D4C4846414600F0D7FD01F097F8139EF6
:10473000109F119A77600D9D0C9F32601521782291
:10474000002360613046B760F56031617261337695
:1047500015B0BDE8F08F0022304B2046294601F00D
:104760002DF818BB24A3D3E900232046294601F0E5
:1047700025F820BB22A3D3E900232046294601F0D7
:104780001DF8031C18BF012301249C4020461293EE
:1047900000F03CFD02460B462046CDE9002300F028
:1047A00025FDDDE90023CDE90A010FE71C4C0023BC
:1047B0000321CDE90A341A461291234606E7194C23
:1047C00000230221CDE90A341A4612912346FDE660
:1047D000A94604F1004899E70000000080842E41BA
:1047E0000000000000205C400000000000206C4041
:1047F0009EE7799EE779EE3F00000000003091408F
:10480000000000000030A1400000304000004040A7
:1048100000002E4000408F40100B001000308140FF
:10482000000020400000104000407F402DE9F04390
:1048300089B0024604460B4601A80D46FFF794FED8
:10484000039E1EB9032009B0BDE8F08306990498C1
:10485000059B029A9DF81C704FEA013808EB00583E
:104860009B0301991B4808F5000803F5F653023332
:10487000D20008F2244803EB471702EBC139FFF7D7
:1048800015FB4046FFF712FB0320FFF70FFB3846EE
:10489000FFF70CFBF00000F500400130FFF706FBCE
:1048A0004846FFF703FB0C4B0C4901E0013B0ED0DF
:1048B00091F8A820002AF9D02046294600F0CEFF22
:1048C000074B024600201A6109B0BDE8F0830220C0
:1048D000B9E700BF0500580040771B0000400F40BB
:1048E000100B001070B5204ED6E9064518A3D3E989
:1048F00000232046294600F061FF08B1052070BD65
:1049000015A3D3E900232046294600F075FF0028AF
:10491000F4D113A3D3E90023D6E9000100F0DCFCB5
:1049200022462B4600F0D8FCFFF760FD0028E6D1B8
:104930000BA3D3E90023D6E9040100F0CDFC224605
:104940002B4600F0C9FCBDE87040FFF76FBF00BF09
:10495000AE47E17A14AEEF3F295C8FC2F528F03FF5
:104960000000000080842E4120010010054B4FF014
:104970000001012283F82E109A7183F8AB2083F88E
:104980004010F7E700400F400A0A013A062A1FD8F4
:10499000DFE802F0080C101E1E1A0400124A0A205A
:1049A0001A607047114A1A6012207047104A1A6044
:1049B0003F207047C9B2012912D00DD3022907D177
:1049C0000A4A526F1078EBE70A4A1A600A207047C9
:1049D000002002461A607047044AD26E1078DFE762
:1049E000024A126F1078DBE7A001001040010010AE
:1049F0005401001094010010054B064A10B4012028
:104A000000244FF000411C60586010BC11607047DA
:104A1000400B001000E100E084B008B50DF1080E75
:104A20008EE80F00FFF7ACF90D4B02221A70FCF76D
:104A300065FE0028FBD1102302AA0521FDF75EFBCD
:104A4000FCF75CFE0028FBD1039B069A0521FDF7CD
:104A500055FBFFF79DF9BDE8084004B0704700BF63
:104A6000880B0010024A026000228260704700BF7B
:104A7000DDCCBBAA84B010B588B00BAC84E80E00C6
:104A80000A4A0C9B0392012206920492013302AA65
:104A90000593009203AB8DF808000FCBFFF7BCFF26
:104AA00008B0BDE8104004B0704700BFDDCCBBAA21
:104AB00084B010B588B00C4C03940AAC84E80F00A5
:104AC000FFF77EFC0B9B094A009201330321302241
:104AD00005930691049203AB0FCBFFF79DFF08B03F
:104AE000BDE8104004B07047DDCCBBAA100B00102D
:104AF00000B589B0084B0393002102224FF4804394
:104B0000049305910692009003AB0FCBFFF784FF4F
:104B100009B05DF804FB00BFDDCCBBAA08B50248B4
:104B2000FEF7A4F9C0B208BDE801001038B50024B2
:104B300025460648FEF79AF9C0B2A0400834202C5A
:104B400045EA0005F5D1284638BD00BFE801001050
:104B50002DE9F0430024C3B0074625463048FEF750
:104B600085F9C0B2A0400834202C45EA0005F5D1F3
:104B70002C4B9D4201D0FFF7F9FE00252C4628481A
:104B8000FEF774F9C0B2A8400835202D44EA0004AD
:104B9000F5D100252E462248FEF768F9C0B2A8409C
:104BA0000835202D46EA0006F5D10025A8461C4808
:104BB000FEF75CF9C0B2A8400835202D48EA00088D
:104BC000F5D1B8F1000F28D10025A8461448FEF70A
:104BD0004DF9C0B2A8400835202D48EA0008F5D1AB
:104BE000E94664B107340DEB0405E9460DF107040D
:104BF0000B48FEF73BF904F8010FAC42F8D14946E7
:104C00004FF484723846C9F80080C9F8046000F097
:104C1000C5FF384643B0BDE8F083FFF7A7FED3E7F2
:104C2000E8010010DDCCBBAA084B10B501220446F8
:104C300039205A60FCF72EF83920FCF73FF800289D
:104C4000FAD12046BDE81040FFF762BB400B0010D0
:104C50002DE9F041A248ADF5067DFEF79FF800284A
:104C600033D1A04D2B689F4963B9FFF79FF82B689C
:104C700023B99D4B4FF00042C3F880200DF5067D0F
:104C8000BDE8F0810879994C013B01220B6082401C
:104C9000236896491342FBD00B6803F01F031F2BB8
:104CA00057D0934B53F82000FFF722FF2B79216850
:104CB0008C4801229A400133DBB2052B21EA020223
:104CC00008BF002322600371CFE744AC854D204626
:104CD000FFF73EFF2F6894E8480027BB462B66D0BD
:104CE0003F2B00F08380412B00F0A380532B00F07A
:104CF000EA80522B00F0DC80432B00F09480542B90
:104D00003CD001273FAC01367A4B41963F93429706
:104D100040973EAE94E80F008DF8F870009626613B
:104D2000FFF77AFE9EE7532B17D100272F603FAC89
:104D3000012301366F4A41963F92429340933EAE23
:104D400094E80F00009626618DF8F870FFF764FE76
:104D500088E7FFF725F82879A3E70122013665499E
:104D600041963FAB3F91429240923EAC0FCB06251D
:104D700000948DF8F850FFF74FFE7FE7237A002B61
:104D800000F09380FFF752F83FAC01230136594AF7
:104D900041963F92429340933EAE94E80F00002725
:104DA000009626618DF8F870FFF736FE5AE7A06886
:104DB00000F01CFA46A3D3E9002300F0B7FB4E4BEA
:104DC0000136C3E90401FFF78DFD3FAC4196012395
:104DD0003EAE484A3F924293409300968DF8F800C9
:104DE00094E80F002661FFF717FE3BE70DF1FC0E7C
:104DF000012301363F4A41963F92429340933EAE93
:104E00009EE80F000096CEF810608DF8F870FFF75E
:104E100003FE48A9F822684600F0C0FE94E80F009F
:104E2000FFF746FE1EE7237A002B49D0FEF7ECFF82
:104E3000AAE70DF1FC0E012301362E4A41963F925E
:104E40003EAE429340939EE80F000096CEF810606D
:104E50008DF8F870D4F80C80FFF7DEFDA3682B60A6
:104E60002F71FEF79DFF244B1BA1D1E90001D3E96F
:104E7000062300F05BFB00F0F1FC00F0B7F90646FA
:104E800040460F4600F0B2F900221C4B00F04EFBEA
:104E900002460B463046394600F01EFA00F0B6FCDA
:104EA000FFF7C2FEFEF782FFDCE6FEF7B5FF6BE719
:104EB000A3682B604FF0FF302F71FFF7B5FE36E788
:104EC000FEF79AFF60E7062731E700BFAFF30080E7
:104ED0000000000080842E410000000060E3A64135
:104EE000E8010010480B001000E100E0400B00104A
:104EF000D460001ADDCCBBAA2001001000408F4016
:104F000008B50D4CFEF744FFFEF74AFF0B48FEF7CD
:104F1000F5FF0121607BFCF79DFE0948FEF7EEFFDF
:104F2000FEF744FFFEF750FFFFF792FE0121607B82
:104F3000FCF736FBF8E700BFE8010010E860001A54
:104F40000061001A704700BF704700BF0148FDF7BD
:104F5000F5BC00BFE80100100148FEF7ADB800BF86
:104F6000E8010010AFF3008081F0004102E000BFD3
:104F700083F0004330B54FEA41044FEA430594EA19
:104F8000050F08BF90EA020F1FBF54EA000C55EA54
:104F9000020C7FEA645C7FEA655C00F0E2804FEA25
:104FA0005454D4EB5555B8BF6D420CDD2C4480EA07
:104FB000020281EA030382EA000083EA010180EA37
:104FC000020281EA0303362D88BF30BD11F0004F85
:104FD0004FEA01314FF4801C4CEA113102D04042BB
:104FE00061EB410113F0004F4FEA03334CEA1333F6
:104FF00002D0524263EB430394EA050F00F0A7800E
:10500000A4F10104D5F1200E0DDB02FA0EFC22FA08
:1050100005F2801841F1000103FA0EF2801843FAFC
:1050200005F359410EE0A5F120050EF1200E012AED
:1050300003FA0EFC28BF4CF0020C43FA05F3C0182B
:1050400051EBE37101F0004507D54FF0000EDCF1A4
:10505000000C7EEB00006EEB0101B1F5801F1BD34D
:10506000B1F5001F0CD349085FEA30004FEA3C0C51
:1050700004F101044FEA445212F5800F80F09A8047
:10508000BCF1004F08BF5FEA500C50F1000041EB4B
:10509000045141EA050130BD5FEA4C0C404141EB4F
:1050A000010111F4801FA4F10104E9D191F0000F76
:1050B00004BF01460020B1FA81F308BF2033A3F1F9
:1050C0000B03B3F120020CDA0C3208DD02F1140CF0
:1050D000C2F10C0201FA0CF021FA02F10CE002F12B
:1050E0001402D8BFC2F1200C01FA02F120FA0CFC24
:1050F000DCBF41EA0C019040E41AA2BF01EB04516D
:10510000294330BD6FEA04041F3C1CDA0C340EDC6A
:1051100004F11404C4F1200220FA04F001FA02F3AD
:1051200040EA030021FA04F345EA030130BDC4F16B
:105130000C04C4F1200220FA02F001FA04F340EA60
:105140000300294630BD21FA04F0294630BD94F011
:10515000000F83F4801306BF81F480110134013DF8
:105160004EE77FEA645C18BF7FEA655C29D094EA69
:10517000050F08BF90EA020F05D054EA000C04BFE7
:105180001946104630BD91EA030F1EBF00210020D2
:1051900030BD5FEA545C05D14000494128BF41F071
:1051A000004130BD14F580043CBF01F5801130BDD5
:1051B00001F0004545F0FE4141F470014FF0000060
:1051C00030BD7FEA645C1ABF194610467FEA655C11
:1051D0001CBF0B46024650EA013406BF52EA0335B3
:1051E00091EA030F41F4002130BD00BF90F0000FA1
:1051F00004BF0021704730B54FF4806404F13204DD
:105200004FF000054FF0000150E700BF90F0000F95
:1052100004BF0021704730B54FF4806404F13204BC
:1052200010F0004548BF40424FF000013EE700BF8C
:1052300042004FEAE2014FEA31014FEA02701FBF1C
:1052400012F07F4393F07F4F81F06051704792F0EE
:10525000000F14BF93F07F4F704730B54FF4607468
:1052600001F0004521F0004120E700BF50EA0102B3
:1052700008BF704730B54FF000050AE050EA010260
:1052800008BF704730B511F0004502D5404261EBD0
:1052900041014FF4806404F132045FEA915C3FF411
:1052A000DCAE4FF003025FEADC0C18BF03325FEAAA
:1052B000DC0C18BF033202EBDC02C2F1200300FA5F
:1052C00003FC20FA02F001FA03FE40EA0E0021FA84
:1052D00002F11444C1E600BF70B54FF0FF0C4CF46E
:1052E000E06C1CEA11541DBF1CEA135594EA0C0F24
:1052F00095EA0C0F00F0DEF82C4481EA030621EA5F
:105300004C5123EA4C5350EA013518BF52EA033599
:1053100041F4801143F4801338D0A0FB02CE4FF04B
:105320000005E1FB02E506F00042E0FB03E54FF07B
:105330000006E1FB03569CF0000F18BF4EF0010E73
:10534000A4F1FF04B6F5007F64F5407404D25FEA6F
:105350004E0E6D4146EB060642EAC62141EA555122
:105360004FEAC52040EA5E504FEACE2EB4F1FD0C64
:1053700088BFBCF5E06F1ED8BEF1004F08BF5FEAE2
:10538000500E50F1000041EB045170BD06F0004694
:1053900046EA010140EA020081EA0301B4EB5C0441
:1053A000C2BFD4EB0C0541EA045170BD41F4801139
:1053B0004FF0000E013C00F3AB8014F1360FDEBF5E
:1053C000002001F0004170BDC4F10004203C35DA3A
:1053D0000C341BDC04F11404C4F1200500FA05F3BD
:1053E00020FA04F001FA05F240EA020001F000425E
:1053F00021F0004110EBD37021FA04F642EB0601D4
:105400005EEA430E08BF20EAD37070BDC4F10C04FD
:10541000C4F1200500FA04F320FA05F001FA04F2C1
:1054200040EA020001F0004110EBD37041F10001AD
:105430005EEA430E08BF20EAD37070BDC4F12005B8
:1054400000FA05F24EEA020E20FA04F301FA05F220
:1054500043EA020321FA04F001F0004121FA04F2C8
:1054600020EA020000EBD3705EEA430E08BF20EA98
:10547000D37070BD94F0000F0FD101F000464000D2
:1054800041EB010111F4801F08BF013CF7D041EA54
:10549000060195F0000F18BF704703F00046520058
:1054A00043EB030313F4801F08BF013DF7D043EA29
:1054B0000603704794EA0C0F0CEA135518BF95EADF
:1054C0000C0F0CD050EA410618BF52EA4306D1D166
:1054D00081EA030101F000414FF0000070BD50EA85
:1054E000410606BF1046194652EA430619D094EA0F
:1054F0000C0F02D150EA013613D195EA0C0F05D1F9
:1055000052EA03361CBF104619460AD181EA03014C
:1055100001F0004141F0FE4141F470014FF0000004
:1055200070BD41F0FE4141F4780170BD70B54FF09F
:10553000FF0C4CF4E06C1CEA11541DBF1CEA13551F
:1055400094EA0C0F95EA0C0F00F0A7F8A4EB050401
:1055500081EA030E52EA03354FEA013100F08880F8
:105560004FEA03334FF0805545EA131343EA1263C1
:105570004FEA022245EA111545EA10654FEA002676
:105580000EF000419D4208BF964244F1FD0404F52F
:10559000407402D25B084FEA3202B61A65EB03058B
:1055A0005B084FEA32024FF480104FF4002CB6EB48
:1055B000020E75EB030E22BFB61A754640EA0C00C8
:1055C0005B084FEA3202B6EB020E75EB030E22BF08
:1055D000B61A754640EA5C005B084FEA3202B6EB49
:1055E000020E75EB030E22BFB61A754640EA9C0008
:1055F0005B084FEA3202B6EB020E75EB030E22BFD8
:10560000B61A754640EADC0055EA060E18D04FEA95
:10561000051545EA16754FEA06164FEAC30343EA35
:1056200052734FEAC2025FEA1C1CC0D111F4801F02
:105630000BD141EA00014FF000004FF0004CB6E7FB
:1056400011F4801F04BF01430020B4F1FD0C88BF9A
:10565000BCF5E06F3FF6AFAEB5EB030C04BFB6EBA5
:10566000020C5FEA500C50F1000041EB045170BD98
:105670000EF0004E4EEA113114EB5C04C2BFD4EBC5
:105680000C0541EA045170BD41F480114FF0000E49
:10569000013C90E645EA060E8DE60CEA135594EAC5
:1056A0000C0F08BF95EA0C0F3FF43BAF94EA0C0FC8
:1056B0000AD150EA01347FF434AF95EA0C0F7FF43D
:1056C00025AF104619462CE795EA0C0F06D152EA91
:1056D00003353FF4FDAE1046194622E750EA410675
:1056E00018BF52EA43067FF4C5AE50EA41047FF486
:1056F0000DAF52EA43057FF4EBAE12E74FF0FF3CEB
:1057000006E000BF4FF0010C02E000BF4FF0010CBB
:105710004DF804CD4FEA410C7FEA6C5C4FEA430C34
:1057200018BF7FEA6C5C1BD001B050EA410C0CBF83
:1057300052EA430C91EA030F02BF90EA020F0020E5
:10574000704710F1000F91EA030F58BF994208BF4C
:1057500090422CBFD8176FEAE37040F00100704709
:105760004FEA410C7FEA6C5C02D150EA013C07D160
:105770004FEA430C7FEA6C5CD6D152EA033CD3D0AB
:105780005DF8040B704700BF8446104662468C46A5
:105790001946634600E000BF01B5FFF7B7FF0028D8
:1057A00048BF10F1000F01BD4DF808EDFFF7F4FF01
:1057B0000CBF012000205DF808FB00BF4DF808ED8C
:1057C000FFF7EAFF34BF012000205DF808FB00BFAF
:1057D0004DF808EDFFF7E0FF94BF012000205DF8D1
:1057E00008FB00BF4DF808EDFFF7CEFF94BF012086
:1057F00000205DF808FB00BF4DF808EDFFF7C4FF7F
:1058000034BF012000205DF808FB00BF4FEA4102D1
:1058100012F5001215D211D56FF47873B3EB625202
:1058200012D94FEAC12343F0004343EA505311F029
:10583000004F23FA02F018BF404270474FF00000BB
:10584000704750EA013005D111F0004008BF6FF0F9
:10585000004070474FF00000704700BF4A0011D26F
:1058600012F5001211D20DD56FF47873B3EB6252BA
:105870000ED44FEAC12343F0004343EA505323FAC6
:1058800002F070474FF00000704750EA013002D13B
:105890004FF0FF3070474FF00000704753B94AB9DE
:1058A000002908BF00281CBF4FF0FF314FF0FF3028
:1058B00000F072B9ADF1080C6DE904CE00F006F805
:1058C000DDF804E0DDE9022304B070472DE9F04F74
:1058D000099E964604460D46002B40F0D5808A422C
:1058E00044D9B2FA82F757B1C7F1200420FA04F480
:1058F000B94044EA010502FA07FE00FA07F44FEA4C
:105900001E4C1FFA8EF3B5FBFCF80CFB1851250C4E
:1059100008FB03F945EA014189450AD911EB0E015B
:1059200008F1FF3006D2894504D9A8F1020071447C
:1059300000E04046C9EB0101A4B2B1FBFCF50CFB51
:1059400015116B4344EA0142934209D912EB0E024E
:1059500005F1FF3105D2934203D9A91E724400E03C
:10596000294641EA0040D31A002184E01AB94FF0D9
:10597000010EBEFBF2FEBEFA8EF71FB9CEEB0100A0
:10598000012142E0C7F1200421FA04F80EFA07FED3
:1059900020FA04F4B94044EA01054FEA1E4C00FA2B
:1059A00007F4B8FBFCF91FFA8EF00CFB19882A0CDF
:1059B00009FB00F142EA084399420AD913EB0E03AE
:1059C00009F1FF3806D2994204D9A9F102087344BB
:1059D00000E0C8465B1AADB2B3FBFCF90CFB19330F
:1059E00009FB00F245EA034082420AD910EB0E009F
:1059F00009F1FF3106D2824204D9A9F102017044B3
:105A000000E04946801A41EA08414FEA1E4C1FFA5D
:105A10008EF2B0FBFCF8250C0CFB180008FB02F31F
:105A200045EA004083420AD910EB0E0008F1FF3529
:105A300006D2834204D9A8F10205704400E045462D
:105A4000C01AA4B2B0FBFCF80CFB180008FB02F271
:105A500044EA00439A420AD913EB0E0308F1FF30DF
:105A600006D29A4204D9A8F10200734400E04046ED
:105A70009B1A40EA0540002E00F08C80FB4033600A
:105A800000237360BDE8F08F8B4205D9002E7CD0D7
:105A900086E80300002179E0B3FA83F77FB98B42EF
:105AA00001D3824205D8841A61EB030101200D461F
:105AB00000E03846002E6CD086E8300062E0C7F186
:105AC000200EBB4022FA0EF521FA0EF820FA0EF451
:105AD0001D43B94021434FEA154900FA07FAABB21A
:105AE000B8FBF9F04FEA114B09FB108C00FB03F4F3
:105AF0004BEA0C4C644502FA07F20AD91CEB050C80
:105B000000F1FF3806D2644504D9A0F10208AC4484
:105B100000E08046C4EB0C0C89B2BCFBF9FB09FB2E
:105B20001BCC0BFB03F341EA0C44A34209D96419D3
:105B30000BF1FF3006D2A34204D9ABF102002C4492
:105B400000E0584640EA0840A0FB0289E41A4C45B0
:105B5000C446494602D308D1C24505D2B8EB020C6F
:105B600069EB0501013800E0214696B1BAEB0C0360
:105B700064EB010404FA0EFEFB404EEA0303FC4012
:105B800086E818000021BDE8F08F31460846BDE8E0
:105B9000F08F3146BDE8F08F704700BF844641EA80
:105BA000000313F003036DD1403A41D351F8043B95
:105BB00040F8043B51F8043B40F8043B51F8043BE7
:105BC00040F8043B51F8043B40F8043B51F8043BD7
:105BD00040F8043B51F8043B40F8043B51F8043BC7
:105BE00040F8043B51F8043B40F8043B51F8043BB7
:105BF00040F8043B51F8043B40F8043B51F8043BA7
:105C000040F8043B51F8043B40F8043B51F8043B96
:105C100040F8043B51F8043B40F8043B51F8043B86
:105C200040F8043B51F8043B40F8043B403ABDD2F5
:105C3000303211D351F8043B40F8043B51F8043B97
:105C400040F8043B51F8043B40F8043B51F8043B56
:105C500040F8043B103AEDD20C3205D351F8043B26
:105C600040F8043B043AF9D2043208D0D2071CBFF2
:105C700011F8013B00F8013B01D30B88038060461B
:105C8000704700BF082A13D38B078DD010F0030391
:105C90008AD0C3F10403D21ADB071CBF11F8013B01
:105CA00000F8013B80D331F8023B20F8023B7BE750
:105CB000043AD9D3013A11F8013B00F8013BF9D27B
:105CC0000B7803704B7843708B7883706046704715
:105CD00070B4840746D0541E002A41D0CDB203468A
:105CE00002E0621EE4B3144603F8015B9A07F8D1A0
:105CF000032C2ED9CDB245EA05250F2C45EA0545E2
:105D000019D903F110022646103E0F2E42F8105CFE
:105D100042F80C5C42F8085C42F8045C02F11002A4
:105D2000F2D8A4F1100222F00F0204F00F04103296
:105D3000032C13440DD91E462246043A032A46F882
:105D4000045BFAD8221F22F003020432134404F049
:105D500003042CB1C9B21C4403F8011BA342FBD1BC
:105D600070BC704714460346C2E700BF20F0030131
:105D700010F00300C0F1000051F8043B00F1040CE6
:105D80004FEACC0C6FF000021CBF22FA0CF2134356
:105D90004FF0010C4CEA0C2C4CEA0C4CA3EB0C021F
:105DA00022EA030212EACC1204BF51F8043B043089
:105DB000F4D0C2F1000102EA0102B2FA82F2C2F1A9
:105DC0001F0200EBD200704701020408000005002A
:105DD0000A00200024000900400040000500600087
:105DE000A600040001000000020000000400000002
:105DF0000800000080000000000100000002000018
:105E000001418100636F6E6669677572696E672014
:105E1000656E64706F696E740A0000002E2E2E206D
:105E2000646F6E650A00000063616C6C696E6720C8
:105E3000555342436F6E6E6563740A00686920664D
:105E4000726F6D207573625F696E69740A0000007D
:105E50007365742063757272656E74206D6F64650E
:105E600020646F6E650A000048414C20696E6974B9
:105E700020646F6E650000002A2A20496E697469EB
:105E8000616C697A696E6720555342206465766952
:105E900063650A00696661636520726573657420D5
:105EA000646F6E6500FFFFFF0030001000280010D7
:105EB000002D00108021001000200010002C001088
:105EC000456E746572696E672048414C5F52657318
:105ED00065740A0031206F6B0A00000032206F6B7E
:105EE0000A00000033206F6B0A00000034206F6B43
:105EF0000A00000035206F6B0A00000036206F6B2F
:105F00000A0000002E2E2E6F6B0A0000436C6561A4
:105F100072696E6720696E746572727570730A00BB
:105F2000312F35206F6B0A00322F35206F6B0A003E
:105F3000332F35206F6B0A00342F35206F6B0A002A
:105F40002E2E2E6F6B205B312F335D0A0000000078
:105F50002E2E2E6F6B205B322F335D0A0000000067
:105F60002E2E2E6F6B205B332F335D0A00FFFFFF59
:105F70000060004000700040636F6E6E656374697E
:105F80006E67205553420A0068692066726F6D2063
:105F900068616C5F696E69740A000000636F726506
:105FA00020776173206E6F7420656E61626C65642A
:105FB0000A000000656E61626C696E67205553428D
:105FC00020504C4C0A00000077616974696E6720AC
:105FD000666F7220504C4C206C6F636B0A0000009F
:105FE00055534220504C4C206C6F636B6564210A02
:105FF00000000000656E61626C696E672055534257
:10600000206261736520636C6F636B0A000000009F
:106010006261736520636C6F636B20656E61626C97
:106020006564210A00000000726573657474696E0E
:106030006720636F6E74726F6C6C65720A0000008B
:106040002E2E2E206F6B0A007265736574206669B0
:106050006E69736865640A0073657474696E67209D
:106060004F54472073746174650A0000696E697447
:10607000696174696E672048414C2072657365746C
:106080000A0000002E2E2E20646F6E65210A00FF8C
:10609000A1200000000002000000002000400020BD
:1060A0000080002000C00020000008100008040943
:1060B000020A050B7374617274696E672075702033
:1060C0004D3020636F72650A00FFFFFF000804096E
:1060D000020A050B00000020004000200080002084
:1060E00000C000200000081053657475704861728C
:1060F00064776172652063616C6C65640A000000FE
:106100005553425F496E697420646F6E650A0000E2
:08611000BCF7FF7F0100000055
:1061180000000020FFFFFFFFAA605452278026409E
:1061280000000000000038400000000000689740B0
:10613800000000000000F03F1201000202000040D1
:10614800C91F4720010001020001000009023E00AA
:1061580002010080FA09040000010202000005247F
:106168000010010424020605240600010705810326
:1061780008000409040100020A00000007050302E0
:106188000002010705820200020100000A0600025F
:1061980000000040010000000A070A000100010099
:1061A800FA000000E4010010DC010010B801001042
:1061B800240332003100200063006D0020004800F5
:1061C8004900200052006500630065006900760000
:1061D8006500720008034E005800500004030904CB
:1061E8000002000200030002000108000000000095
:0C61F8000000000000000000000000009B
:040000051A0001D507
:00000001FF
